:10000000283084005830A0008001840AA00B042806
:10001000103095002730960000308E0000308F00A1
:10002000013090000B30970007309F008316FF309F
:10003000850083128316CF30860083120C1D1E2884
:100040000C116400A914A9182915A91C2911A911BA
:1000500029192916291D2912851B2F282912291E25
:100060003228A91529192916291D2912051B3928F5
:100070002912291E3C28A915A9192915A91D2911DC
:100080002919A916291DA912291F47282911A91ABA
:100090002917A91E2913291D5228A91B5228AA0F66
:1000A0005228AB0A2919A917291DA91300302B02C0
:1000B00003196128A00020092B05A006A01B6628B3
:1000C000682801302A02031C66286828291169283B
:1000D000291529198616291D8612A9182915A91C62
:1000E0002911861A74282911291D8B2827302D02E1
:1000F00003198128A00020092D05A006A01B862831
:100100008A280F302C02031C86288A28AC0F8928E5
:10011000AD0A29118F280030AC000030AD00291D38
:1001200095280030AA000030AB00A9182915A91C99
:100130002911861A9C282911061E9F2829112E187C
:10014000A5283130AF000030B0002E142919BD2889
:10015000003030020319B328A00020093005A006A2
:10016000A01BB828BC2831302F02031CB828BC289B
:10017000AF0FBB28B00A2915C1280030AF000030EE
:10018000B000291DD828003032020319CE28A00063
:1001900020093205A006A01BD328D7283130310210
:1001A000031CD328D728B10FD628B20A2911DC287E
:1001B0000030B1000030B20029190616291D0612C0
:1001C0008A011E28FF3FFF3FFF3FFF3FFF3FFF3FEA
:1001D000FF3FFF3FFF3FFF3FFF3FFF3FFF3FFF3F2F
:1001E000FF3FFF3FFF3FFF3FFF3FFF3FFF3FFF3F1F
:1001F000FF3FFF3FFF3FFF3FFF3FFF3FFF3FFF3F0F
:10020000FF3FFF3FFF3FFF3FFF3FFF3FFF3FFF3FFE
:02400E0050035D
:10420000FF00FF00FF00FF00FF00FF00FF00FF00B6
:10421000FF00FF00FF00FF00FF00FF00FF00FF00A6
:10422000FF00FF00FF00FF00FF00FF00FF00FF0096
:10423000FF00FF00FF00FF00FF00FF00FF00FF0086
:10424000FF00FF00FF00FF00FF00FF00FF00FF0076
:10425000FF00FF00FF00FF00FF00FF00FF00FF0066
:10426000FF00FF00FF00FF00FF00FF00FF00FF0056
:10427000FF00FF00FF00FF00FF00FF00FF00FF0046
:10428000FF00FF00FF00FF00FF00FF00FF00FF0036
:10429000FF00FF00FF00FF00FF00FF00FF00FF0026
:1042A000FF00FF00FF00FF00FF00FF00FF00FF0016
:1042B000FF00FF00FF00FF00FF00FF00FF00FF0006
:1042C000FF00FF00FF00FF00FF00FF00FF00FF00F6
:1042D000FF00FF00FF00FF00FF00FF00FF00FF00E6
:1042E000FF00FF00FF00FF00FF00FF00FF00FF00D6
:1042F000FF00FF00FF00FF00FF00FF00FF00FF00C6
:00000001FF
